:020000040800F2
:10000000005000202D0E0008890200088B02000815
:100010008D0200088F020008910200080000000015
:100020000000000000000000000000009302000833
:1000300095020008000000009702000899020008DD
:10004000750E0008750E0008750E0008750E000884
:10005000750E0008750E0008750E0008750E000874
:10006000750E0008750E0008750E0008750E000864
:10007000750E0008750E0008750E0008750E000854
:10008000750E0008750E0008750E0008750E000844
:10009000750E0008750E0008750E0008750E000834
:1000A000750E0008750E0008750E0008750E000824
:1000B000750E0008750E0008750E0008750E000814
:1000C000750E0008750E0008750E0008750E000804
:1000D000750E0008750E0008750E0008750E0008F4
:1000E000750E0008750E0008750E0008000000006F
:1000F0000000000000000000000000000000000000
:0C01000000000000000000005FF808F1A3
:10010C0010B5054C237833B9044B13B10448AFF345
:10011C0000800123237010BD0C00002000000000A3
:10012C00C00E000808B5034B1BB103490348AFF3DD
:10013C00008008BD0000000010000020C00E000868
:10014C0030B589B000240494059406940794174B99
:10015C009A6942F020029A619A6902F02002019297
:10016C00019A9A6942F004029A619A6902F00402B7
:10017C000292029A9A6942F008029A619B6903F012
:10018C0008030393039B0A4D22461F21284600F0C7
:10019C00E3FD1F2304930123059306940223079385
:1001AC0004A9284600F0ECFC09B030BD0010024058
:1001BC000008014008B50948094B0360102343604F
:1001CC0000238360C36003614361037643768376C7
:1001DC00C3760377437700F0C3F808BD28000020EE
:1001EC000064004070B590B00024089409940B94FE
:1001FC000C9401940294039404940594012506959F
:10020C004FF4803307930A9502260D960E934FF404
:10021C00E0130F9306A800F0BDF90F23019302968B
:10022C00039404940594294601A800F0F3FB10B044
:10023C0070BD000008B500F05FF9FFF7D3FFFFF7C2
:10024C007FFFFFF7B7FF0C4BDA680022DA600A4C2D
:10025C00E36883F00103E360C82000F071F9E36800
:10026C0083F00803E360E36883F01003E36042F279
:10027C00107000F065F9EAE7000801407047FEE7EE
:10028C00FEE7FEE7FEE770477047704708B500F0E1
:10029C0045F908BD82B00E4B9A6942F001029A6191
:1002AC009A6902F001020092009ADA6942F08052D7
:1002BC00DA61DB6903F080530193019B054A5368B3
:1002CC0023F0E06343F08063536002B0704700BFDB
:1002DC00001002400000014010B586B000230293CC
:1002EC0003930493059302681A4B9A4201D006B00B
:1002FC0010BD03F5D633DA6942F00072DA61DA69BF
:10030C0002F000720092009A9A6942F008029A6117
:10031C009B6903F008030193019B4FF480730293D4
:10032C000D4C02A9204600F02BFC4FF400730293F5
:10033C00022303930323059302A9204600F020FC1B
:10034C00064A536823F4C04343F0E06343F480430C
:10035C005360CCE700640040000C014000000140F9
:10036C00002800F0A18038B5044690F82030D3B1B5
:10037C002268136823F00203136000F0DBF80546D3
:10038C0023685A6812F0020F10D000F0D3F8401B0B
:10039C000A28F5D9636A43F400336362052384F8B1
:1003AC002030012038BDFFF797FFE1E71A6842F0D3
:1003BC0001021A6000F0BEF8054623685A6812F074
:1003CC00010F0DD100F0B6F8401B0A28F5D9636A6D
:1003DC0043F400336362052384F820300120E1E705
:1003EC00227E012A3DD01A6822F080021A60637EB8
:1003FC00012B3BD02268136823F040031360A37ECB
:10040C00012B39D02268136823F020031360E37E9C
:10041C00012B37D02268136843F010031360237F3D
:10042C00012B35D02268136823F008031360637F17
:10043C00012B33D02268136823F004031360A368E4
:10044C00E268134322691343626913436268013AF9
:10045C0021681343CB6100206062012384F82030B3
:10046C00A0E71A6842F080021A60C0E7226813689D
:10047C0043F040031360C2E72268136843F0200383
:10048C001360C4E72268136823F010031360C6E7F7
:10049C002268136843F008031360C8E722681368E6
:1004AC0043F004031360CAE70120704710B50446FB
:1004BC000E4B18784FF47A73B3FBF0F30C4A1068B8
:1004CC00B0FBF3F000F094FC68B90F2C01D90120BB
:1004DC000AE0002221464FF0FF3000F055FC054B9E
:1004EC001C60002000E0012010BD00BF00000020B7
:1004FC00080000200400002008B5074A136843F0E8
:10050C0010031360032000F02DFC0020FFF7CEFF3A
:10051C00FFF7C0FE002008BD00200240034A11680E
:10052C00034B1B780B441360704700BF5000002036
:10053C0000000020014B1868704700BF50000020DD
:10054C0038B50446FFF7F6FF0546B4F1FF3F02D07D
:10055C00044B1B781C44FFF7EDFF401BA042FAD361
:10056C0038BD00BF0000002082B0084B1B68084A51
:10057C00A2FB03235B0A00FB03F0019000BF019B6D
:10058C005A1E0192002BF9D102B0704708000020CE
:10059C00D34D6210002800F0F18170B582B0044692
:1005AC00036813F0010F2CD0AA4B5B6803F00C030B
:1005BC00042B1DD0A74B5B6803F00C03082B12D047
:1005CC006368B3F5803F41D0002B55D103F18043D4
:1005DC0003F504331A6822F480321A601A6822F484
:1005EC0080221A6037E09B4B5B6813F4803FE7D0A6
:1005FC00984B1B6813F4003F03D06368002B00F08A
:10060C00BF81236813F0020F75D0924B5B6813F017
:10061C000C0F5FD08F4B5B6803F00C03082B54D08E
:10062C002369002B00F089808B4B01221A60FFF7A5
:10063C0081FF0546874B1B6813F0020F74D1FFF73F
:10064C0079FF401B0228F5D903209EE1814A1368EB
:10065C0043F480331360636843B3FFF76BFF0546C5
:10066C007C4B1B6813F4003FCBD1FFF763FF401B9F
:10067C006428F5D9032088E1B3F5A02F09D0754B78
:10068C001A6822F480321A601A6822F480221A60E6
:10069C00E1E703F18043A3F53C331A6842F480226E
:1006AC001A601A6842F480321A60D4E7FFF742FFEE
:1006BC000546684B1B6813F4003FA2D0FFF73AFFC6
:1006CC00401B6428F5D903205FE1624B5B6813F48F
:1006DC00803FA5D15F4B1B6813F0020F03D0236939
:1006EC00012B40F04F815B4A136823F0F8036169DA
:1006FC0043EAC1031360236813F0080F32D0A369D7
:10070C00002B5BD0554B01221A60FFF713FF0546F7
:10071C00504B5B6A13F0020F21D1FFF70BFF401B0C
:10072C000228F5D9032030E14A4A136823F0F80374
:10073C00616943EAC1031360DDE7474B00221A608D
:10074C00FFF7F8FE0546434B1B6813F0020FD2D09F
:10075C00FFF7F0FE401B0228F5D9032015E101201C
:10076C00FFF702FF236813F0040F00F09780394B5A
:10077C00DB6913F0805F33D1364BDA6942F080527B
:10078C00DA61DB6903F080530193019B0125344B43
:10079C001B6813F4807F25D0E368012B36D0002B27
:1007AC004CD103F1804303F504331A6A22F00102A1
:1007BC001A621A6A22F004021A622CE0274B0022F9
:1007CC001A60FFF7B7FE0546224B5B6A13F0020F67
:1007DC00C8D0FFF7AFFE401B0228F5D90320D4E0A8
:1007EC000025D4E71E4A136843F480731360FFF7A7
:1007FC00A1FE06461A4B1B6813F4807FCCD1FFF781
:10080C0099FE801B6428F5D90320BEE0114A136AB7
:10081C0043F001031362E36873B3FFF78BFE0646E4
:10082C000C4B1B6A13F0020F37D1FFF783FE801BB2
:10083C0041F288339842F3D90320A6E0052B11D05E
:10084C00044B1A6A22F001021A621A6A22F004029C
:10085C001A62E0E70010024000004242800442426B
:10086C00007000404D4B1A6A42F004021A621A6A78
:10087C0042F001021A62CEE7FFF75CFE0646474BD8
:10088C001B6A13F0020F08D0FFF754FE801B41F2D5
:10089C0088339842F3D9032077E0E5B9E369002B5C
:1008AC0072D03E4A526802F00C02082A56D0022B33
:1008BC0017D03B4B00221A60FFF73CFE0446374B27
:1008CC001B6813F0007F47D0FFF734FE001B022893
:1008DC00F5D9032059E0314AD36923F08053D36111
:1008EC00DCE72F4B00221A60FFF724FE05462B4B4A
:1008FC001B6813F0007F06D0FFF71CFE401B02287C
:10090C00F5D9032041E0236AB3F5803F1AD023497F
:10091C004B6823F47413226A606A024313434B60DE
:10092C001F4B01221A60FFF705FE04461B4B1B6888
:10093C0013F0007F0ED1FFF7FDFD001B0228F5D947
:10094C00032022E0154A536823F40033A1680B43BB
:10095C005360DCE7002018E0002016E0012B16D0D5
:10096C000E4B5B6803F48031226A914211D103F47F
:10097C007013626A93420ED1002006E0012070478A
:10098C00012002E0012000E0002002B070BD012037
:10099C00FBE70120F9E70120F7E700BF0010024058
:1009AC006000424210B487B0164C94E80F000DF171
:1009BC00180C0CE90F00238AADF80430124B5B685D
:1009CC0003F00C02082A03D0104807B010BC704783
:1009DC00C3F38342624412F8102C13F4803F0CD002
:1009EC00094B5B68C3F34043634413F8143C07485A
:1009FC0000FB02F0B0FBF3F0E7E7054800FB02F068
:100A0C00E3E700BFD80E00080010024000127A0085
:100A1C0000093D00002800F0A08070B50446534B3F
:100A2C001B6803F007038B420BD2504A136823F068
:100A3C0007030B431360136803F007038B4240F06A
:100A4C008E80236813F0020F17D013F0040F04D01C
:100A5C00474A536843F4E0635360236813F0080F6C
:100A6C0004D0434A536843F460535360404A53687C
:100A7C0023F0F003A068034353600D46236813F082
:100A8C00010F31D06368012B20D0022B25D0384ABE
:100A9C00126812F0020F64D035494A6822F0030242
:100AAC0013434B60FFF746FD0646314B5B6803F082
:100ABC000C036268B3EB820F16D0FFF73BFD801B73
:100ACC0041F288339842F0D9032045E0284A126855
:100ADC0012F4003FE0D101203EE0254A126812F0EA
:100AEC00007FD9D1012037E0204B1B6803F00703AE
:100AFC00AB420AD91D4A136823F007032B4313603A
:100B0C00136803F00703AB422DD1236813F0040FD5
:100B1C0006D0174A536823F4E063E1680B43536033
:100B2C00236813F0080F07D0114A536823F460535D
:100B3C00216943EAC1035360FFF734FF0C4B5B6838
:100B4C00C3F303130B4AD35CD8400B4B18600B4B0D
:100B5C001868FFF7ABFC002070BD01207047012026
:100B6C00FAE70120F8E70120F6E700BF0020024079
:100B7C0000100240EC0E00080800002004000020C9
:100B8C00F0B482B000263546A0E0002A58D0012AE5
:100B9C0010D1CE680EE06A4FBA4251D048D9694F95
:100BAC00BA424DD007F58037BA4249D0A7F5801725
:100BBC00BA4245D0FF2B57D88446FF2B57D8AC00F0
:100BCC00DCF800200F27A74022EA070206FA04F4FB
:100BDC002243CCF800204A6812F0805F75D05A4A44
:100BEC00946944F001049461926902F0010201924B
:100BFC00019AAC08A71C554A52F8272005F00307A8
:100C0C00BF004FF00F0C0CFA07FC22EA0C0C504AF8
:100C1C00904232D002F58062904271D002F580622F
:100C2C0090426FD002F58062904224D0042225E0DD
:100C3C00A7F58017BA4203D007F58037BA42B9D16D
:100C4C008A687AB1012A08D044610826B2E7CE68D6
:100C5C000836AFE7CE680C36ACE704610826A9E786
:100C6C000026A7E70426A5E700F1040CA5E7A5F1EB
:100C7C000804A400A4E7032200E00022BA4042EAE0
:100C8C000C020234314F47F824204A6812F4803F9A
:100C9C003AD0304C22681A4322604A6812F4003F62
:100CAC0038D02C4C62681A4362604A6812F4801F78
:100CBC0036D0284CA2681A43A2604A6812F4001F6E
:100CCC0034D0244CE2681343E36001350B6833FAEB
:100CDC0005F231D00124AC4023409C42F5D14A6846
:100CEC00122AB7D03FF657AF022AB0D07FF64DAFDD
:100CFC00032AB5D0112A7FF45DAFCE68043659E7CC
:100D0C000122BBE70222B9E7124C226822EA030255
:100D1C002260C2E70F4C626822EA03026260C4E7F9
:100D2C000C4CA26822EA0302A260C6E7094CE268F6
:100D3C0022EA0303E360C8E702B0F0BC704700BFCF
:100D4C000000211000003110001002400000014092
:100D5C0000080140000401400AB101617047090418
:100D6C0001617047074AD36823F4E0631B041B0C32
:100D7C00000200F4E060184340F0BF6040F4003023
:100D8C00D060704700ED00E030B4174BDB68C3F364
:100D9C000223C3F10704042C28BF04241D1D062DB7
:100DAC0001D9033B00E000234FF0FF3505FA04F4B2
:100DBC0021EA0401994005FA03F322EA03031943DB
:100DCC00002809DB0901C9B200F1604000F561405F
:100DDC0080F8001330BC704700F00F000901C9B255
:100DEC00024B1954F6E700BF00ED00E014ED00E0F3
:100DFC000138B0F1807F0AD2064B5860064AF021C8
:100E0C0082F823100020986007221A607047012096
:100E1C00704700BF10E000E000ED00E070470000FC
:100E2C00002103E00B4B5B58435004310A480B4B39
:100E3C0042189A42F6D30A4A02E0002342F8043BD5
:100E4C00084B9A42F9D3FFF7E9FF00F00FF8FFF7D0
:100E5C00F1F97047040F0008000000200C0000207E
:100E6C000C00002054000020FEE7000070B50026A6
:100E7C000C4D0D4C641BA410A64209D100F01AF8BD
:100E8C0000260A4D0A4C641BA410A64205D170BD65
:100E9C0055F8043B98470136EEE755F8043B984764
:100EAC000136F2E7FC0E0008FC0E0008FC0E0008F0
:100EBC00000F0008F8B500BFF8BC08BC9E46704790
:0C0ECC00F8B500BFF8BC08BC9E4670479B
:100ED80002030405060708090A0B0C0D0E0F101073
:100EE80001020000000000000000000001020304ED
:040EF80006070809D8
:040EFC0031010008B8
:040F00000D010008D7
:0C0F040001000000100000000024F400B8
:0400000508000E2DB4
:00000001FF
